:1000000042C0A7C15BC05AC059C058C057C056C0F3
:1000100055C054C053C052C051C050C04FC04EC054
:100020004DC04CC04BC04AC049C048C047C046C084
:1000300045C044C0090212000101008019090400F2
:1000400000000000000012011001FF000008C016AF
:10005000DC050401010200010E03550053004200BB
:100060006100730070001C037700770077002E009A
:10007000660069007300630068006C002E00640075
:1000800065000403090411241FBECFEFD4E0DEBFD6
:10009000CDBF11E0A0E0B1E0E2EDF1E102C00590DA
:1000A0000D92A230B107D9F711E0A2E0B1E001C092
:1000B0001D92AC34B107E1F779D889C8A1CFCF93AD
:1000C000DF9360912801635067FD13C08091250183
:1000D000CCE0D0E0C81BD109C45DDE4F8091240183
:1000E0008D3209F457C08091020187FD9BC01092A8
:1000F00028018091000184FF40C0609101016F3FA1
:1001000009F43BC0693008F46FC068506093010186
:100110008091180198E889278093180168E0809100
:10012000020187FD1DC0409126015091270186FFE5
:1001300070C0FA01862FA9E1B1E094919D933196A8
:100140008150D9F7262F215030E02F5F3F4F240FE9
:10015000351F3093270120932601C62FCC5F4FC057
:1001600089E191E0ECD6682F893008F4A1C08FEFC7
:1001700080930101CEE1C093000194E183B18370CB
:1001800031F49150D9F71092290110922301DF9197
:10019000CF910895683009F0AACF83EC80931801BD
:1001A0008AE580930001109202018881807609F02F
:1001B00043C09A81109221018981811147C0109218
:1001C000220121E231E082E03093270120932601D1
:1001D0008F3FA9F19F81911104C09E81981708F467
:1001E000892F8093010183CF109201018091180122
:1001F00098E8892780931801611191CFC4E089E1C3
:1002000091E0A3D0CC3009F4B6CF8FEF80930101F9
:10021000B2CFDA01862FE9E1F1E09D91919381500F
:10022000E1F790CFCE01F8D68F3FF1F0882309F4A3
:100230005ECF109201015BCFCE01DCD4C9CF988193
:1002400097FD16C090E890930201CBCF853091F0D6
:10025000863001F18830D1F0893091F021E231E02F
:100260008A3021F180E0B0CF8EE1809300013FCF52
:100270008E81E8CF9093290121E231E080E0A4CF84
:1002800090932B0121E231E080E09ECF2BE231E020
:1002900081E09ACF8B81813001F18230B1F08330DF
:1002A00051F080E090E49093020192CF81E08CCFF6
:1002B000C82FCC5FA4CF911118C082E890E0909332
:1002C00027018093260184E0EDCF84E390E09093B2
:1002D00027018093260182E1E5CF86E490E09093A8
:1002E00027018093260182E1DDCF913051F09230D9
:1002F000C1F688E590E090932701809326018EE077
:10030000D1CF86E690E090932701809326018CE17F
:10031000C9CFE9E6F0E0808183608083E89A0895A0
:10032000A82FB92F80E090E041E050EA609530E0DE
:1003300009C02D9182279795879510F084279527DE
:10034000305EC8F36F5FA8F30895EADF8D939D9345
:100350000895CF93CFB7CF93C395189BE9F7189B18
:1003600009C0189B07C0189B05C0189B03C0189BA9
:1003700001C0A1C0DF93C0912501DD27C45DDE4F20
:10038000189B02C0DF91EBCF2F930F931F9303B104
:100390002FEF00FB20F94F933F9313B14FEF01274D
:1003A00000FB21F93BE031C04E7F012F13B12160EA
:1003B00028C0102F4D7F2260000003B129C04B7F61
:1003C0002460012F000013B12BC013B1477F2860B8
:1003D0002AC04F7E03B120612CC04F7D13B1206233
:1003E0002FC04F7B03B1206432C0422703B1499331
:1003F0004FEF0000102710FB20F913B11370C9F163
:10040000297F91F2012700FB21F903B1237F89F2B3
:10041000315058F1102710FB22F913B1277E79F2E1
:10042000012700FB23F92F7C81F203B1102710FB79
:1004300024F92F7971F200C013B1012700FB25F9CF
:100440002F7359F200C003B1102710FB26F9223098
:1004500040F200C013B1012700FB27F9243028F631
:100460004F77206813B10000F9CF11E01CBB0027C3
:1004700017C03B503195C31BD04011E01CBB088115
:10048000033CE9F00B34D9F0209123011981110FBD
:100490001213EDCF093641F10D3211F0013E39F75B
:1004A00000932A013F914F911F910F912F91DF915E
:1004B000CCB3C0FD51CFCF91CFBFCF911895209134
:1004C0002A01222379F310912801112311F53430E8
:1004D00012F13093280120932401109125013BE073
:1004E000311B3093250117C00091280101308CF495
:1004F0000AE53091000134FD10C000930001C8E10D
:10050000D1E00FC02795A8F45150A9F4220F0000A4
:10051000F9CF4AE503C042ED01C0432FC4E1D0E06A
:1005200032E014B11360289A14B905B120E413E045
:100530005F93012756E005B9279520F4515021F427
:10054000220FF9CF012756E000003B5A05B9D0F23F
:10055000279528F4515029F4220F0000F9CF0127E4
:1005600056E0279505B920F4515021F4220FF9CF18
:10057000012756E02991332305B921F60C7F10910C
:100580002901110FC651D04005B911F01093230174
:1005900011E01CBB016014B11C7F402F4C7F5F91A8
:1005A00000C000C005B914B945B97CCF682F58E028
:1005B00080E0709148012091470167FD1EC02B9893
:1005C000660F880F1C998F5F2D9A36B5472F4150C3
:1005D00030F096B5931B9217E0F34150D0F72D9869
:1005E00036B5472F415030F096B5931B9217E0F384
:1005F0004150D0F7515009F708952B9AE1CF8EBDA5
:100600000DB407FEFDCF8EB5089521E1969587952F
:10061000779567952A95D1F7209146012617D9F04D
:1006200060934601E0914301F09144018DE4099506
:10063000E0914301F091440180E00995E09143018C
:10064000F0914401809146010995E0914301F091B8
:10065000440180E009940895809145018CBD80910A
:1006600042018DBD08958823C1F0883008F042C052
:1006700026ED32E0309344012093430191E09093C2
:100680004801843039F1D8F0863049F158F187308B
:10069000D1F483E08093470108958FEF92E0909327
:1006A00044018093430181E0809347018093480196
:1006B00082E58093450181E0809342010895823074
:1006C00069F0833099F080E68093470182E080935F
:1006D0004801089588E180934701089580E680935A
:1006E000470108958CE080934701089580E380934B
:1006F000470108952FEF32E03093440120934301E6
:100700001092420191E09093470190934801893003
:1007100039F050F4883061F683E5809345010895FF
:1007200082E58093450108958B3049F08C3009F0C3
:10073000BFCF81E58093450190934201089581E503
:1007400080934501089526B5309148019091470165
:10075000315030F086B5821B8917E0F33150D0F765
:10076000089584B18C6284B92A982D9826B5309169
:100770004801432F90914701415030F086B5821BCC
:100780008917E0F34150D0F72A9A26B5315030F05E
:1007900086B5821B8917E0F33150D0F72A988091F3
:1007A0004301909144018F5F924019F010924601ED
:1007B0000895809145018CBD809142018DBD1092BC
:1007C0004601089584B1837D84B985B1837D85B95F
:1007D0001CBC0895CF93DF93C0E2E0914301F091F8
:1007E00044018CEA0995E0914301F091440183E5CD
:1007F0000995E0914301F091440180E00995D82FDB
:10080000E0914301F091440180E00995D33509F46A
:100810003AC01CBC26B530914801432F9091470146
:10082000415030F086B5821B8917E0F34150D0F774
:100830002A9A26B5432F415030F086B5821B89177E
:10084000E0F34150D0F72A9826B5315030F086B504
:10085000821B8917E0F33150D0F7E0914301F0910A
:10086000440182E0EF3FF80739F0C15009F0B9CFF9
:1008700081E0DF91CF910895809145018CBD8091F9
:1008800042018DBDF2CF80E0DF91CF910895CF92EC
:10089000DF92EF92FF926B017C01B7DED701C601B8
:1008A00081709927AA27BB27880F880F880FE091AE
:1008B0004301F091440180620995D701C60139E0F6
:1008C000B695A795979587953A95D1F7E09143010D
:1008D000F09144010995D701C601B695A795979562
:1008E0008795E0914301F09144010995E09143011E
:1008F000F091440180E0FF90EF90DF90CF90099459
:10090000CF92DF92EF92FF920F931F93CF93DF93DB
:100910006B017C01C42FD22F78DE97018601017014
:10092000112722273327802F880F880F880FE09107
:100930004301F091440180640995D701C60159E053
:10094000B695A795979587955A95D1F7E09143016C
:10095000F09144010995D701C601B695A7959795E1
:100960008795E0914301F09144010995E09143019D
:10097000F09144018C2F0995DD23A9F0CF3789F040
:10098000D6B5CEE1C701B60182DF8F3761F486B5F7
:100990008D1B8D3310F0D6B5C150C111F3CF81E05E
:1009A00003C08FE0B2D080E0DF91CF911F910F9113
:1009B000FF90EF90DF90CF900895CF92DF92EF926B
:1009C000FF920F931F93CF93DF931F92CDB7DEB7A4
:1009D0006B017C01498319DEE0914301F0914401F0
:1009E0008CE40995D701C60179E0B695A79597954E
:1009F00087957A95D1F7E0914301F09144010995EB
:100A0000D701C601B695A79597958795E0914301C3
:100A1000F09144010995E0914301F091440180E097
:100A2000099549814F3FE1F006B51EE1C701B601C6
:100A30002EDF8F3F99F486B5801B8D3310F006B5FD
:100A400011501111F3CF81E00F90DF91CF911F91E1
:100A50000F91FF90EF90DF90CF90089580E0F4CF5A
:100A60008FE053D080E0F0CF1F93CF93DF931F929E
:100A7000CDB7DEB7182FE0914301F091440180EA31
:100A800099830995E0914301F09144019981892F5F
:100A90000995E0914301F0914401812F0995E0917E
:100AA0004301F091440180E00F90DF91CF911F91BD
:100AB00009941F93CF93DF9300D0CDB7DEB7182FE3
:100AC000E0914301F091440180EC6A839983099598
:100AD000E0914301F09144019981892F0995E091BA
:100AE0004301F0914401812F0995E0914301F09178
:100AF00044016A81862F09958EE107D080E00F902E
:100B00000F90DF91CF911F910895882349F030E035
:100B100026B596B5921B9C33E0F33F5F3813F8CFB0
:100B20000895259A23982B9A50E217D05A95E9F701
:100B30000895AC0188E605D0842F03D089E601D062
:100B4000852F0FD028E030E0382780FB869506D02F
:100B50002A95D1F730FB02D000D0689423982B9AC5
:100B600016F02B98239AE0914A01F0914B013197AE
:100B7000F0F72D9AE3B1E3FBE0914A01F0914B01CC
:100B80003197F0F72D98089520ECE7DF46F42A9589
:100B9000E1F780E02AE1E5DF2A95E9F7DECF28E0FA
:100BA00030E0DBDF869587F938272A95D1F7D5DF46
:100BB00027F9322772F3D1DFD0CFDB01742FB9DFF1
:100BC00084E2BFDFE1DF8D937A95D1F70895DB01F1
:100BD000742FAFDF83EFB5DF8DE1B3DF84E6B1DFE4
:100BE0008D91AFDF82E7ADDFCFDF8078D9F77A95DF
:100BF00089F70895CF93DF93EC018981813089F1E2
:100C0000823009F4A8C0833009F45FC08430A1F1B8
:100C1000873009F47FC0853009F4FEC0863009F4BE
:100C20009EC0883009F4D1C0893009F4FAC08A30F6
:100C300009F425C18B3009F451C18C3009F461C12C
:100C40008D3009F473C18E3009F475C18F3009F409
:100C5000F9C0803109F41AC18F3709F434C180E03A
:100C60002BC0329B54C080910301FDDC1092040123
:100C7000419877DD80E020C080910401811110C08F
:100C80005B8140E08A81482B662757FD6095762F6F
:100C900040930D0150930E0160930F01709310016A
:100CA0009F8180E02E81822B90931201809311010D
:100CB00082E0809313018FEF25E031E0309327012C
:100CC00020932601DF91CF910895E0914301F091A7
:100CD00044018A81099580930501E0914301F091D7
:100CE00044018B81099580930601E0914301F091C5
:100CF00044018C81099580930701E0914301F091B3
:100D000044018D8109958093080184E0D5CF85E069
:100D1000AADCACCF80910401811110C05B8140E05E
:100D20008A81482B662757FD6095762F40930D01E9
:100D300050930E0160930F01709310019F8180E02A
:100D40002E81822B909312018093110183E0809376
:100D500013018FEFB1CF36DD419A80E0ADCF8091A6
:100D60000401811110C09B8180E02A81822BAA2777
:100D700097FDA095BA2F80930D0190930E01A0933B
:100D80000F01B09310013C812D81822F8F708093D1
:100D90001601822F807F40E1849FC0011124830FC0
:100DA000911D909315018093140120FD80931701EC
:100DB0009F8180E02E81822B9093120180931101FC
:100DC00081E0809313018FEF77CF8091040181112F
:100DD00010C09B8180E02A81822BAA2797FDA095D5
:100DE000BA2F80930D0190930E01A0930F01B09341
:100DF00010011092150110921401109216019F819A
:100E000080E02E81822B909312018093110184E067
:100E1000809313018FEF50CFDDDC8093050181E0DB
:100E20004BCF81E0809304018A819B81AC81BD819D
:100E300080930D0190930E01A0930F01B0931001C8
:100E400080E03ACF9B8180E02A81822BAA2797FD00
:100E5000A095BA2F80930D0190930E01A0930F01DE
:100E6000B09310019F8180E02E81822B909312011C
:100E70008093110185E0809313018FEF1DCF8A814C
:100E8000809303011092050181E016CF9B8180E0E1
:100E90002A81822BAA2797FDA095BA2F80930D0156
:100EA00090930E01A0930F01B09310019F8180E0F9
:100EB0002E81822B909312018093110186E0809302
:100EC00013018FEFF9CE81E08093050110920601A6
:100ED000109207011092080184E0EECE9B8180E021
:100EE0002A81822B90934B0180934A012A9A229A5D
:100EF00083E00BDE2A98419880E107DE12DE80E075
:100F0000DBCE80EC1EDE80E01CDE8AE0FEDD2A9A6D
:100F100085E0FBDD2A9885E0F8DD84B1837D84B926
:100F200085B1837D85B9419A80E0C6CE2DDE809360
:100F3000050181E0C1CE8A8104DE80E0BDCE0F9341
:100F40001F93CF93DF93582F792F062F20911301F2
:100F5000322F3250323050F0253009F441C00FEFBB
:100F6000802FDF91CF911F910F910895662381F11A
:100F700080910D0190910E01A0910F01B09110018F
:100F8000C52FD72F10E01BC06FDD888380910D0126
:100F900090910E01A0910F01B09110010196A11D39
:100FA000B11D80930D0190930E01A0930F01B0939A
:100FB00010011F5F2196101749F020911301223074
:100FC00019F7BC01CD0163DC8883E0CF083040F61F
:100FD00010921301802FDF91CF911F910F910895EF
:100FE000462F682F80910D0190910E01E6DD8091D2
:100FF0000D0190910E01A0910F01B0911001800F91
:10100000911DA11DB11D80930D0190930E01A09320
:101010000F01B0931001A4CFFF920F931F93CF93B2
:10102000DF93382F792F162F20911301213071F083
:10103000243061F0263009F48BC0FF24FA948F2D00
:10104000DF91CF911F910F91FF900895112309F423
:10105000ABC080910D0190910E01A0910F01B09154
:101060001001C32FD72F00E0F12C4EC020911401A6
:1010700030911501232B09F050C021E04881BC01BB
:10108000CD013EDC20911101309112012150310936
:101090003093120120931101232BE1F410921301DC
:1010A0008091160181FF36C02091170130E08091B8
:1010B0001401909115012817390761F160910D0114
:1010C00070910E0180910F0190911001488175DCA3
:1010D000FF24F39480910D0190910E01A0910F01D6
:1010E000B09110010196A11DB11D80930D01909347
:1010F0000E01A0930F01B09310010F5F219601170D
:1011000009F49DCF20911301213009F4AFCF6881FC
:10111000D0DCB8CFFF24F394DDCF20E04881BC01C0
:10112000CD01EEDB80911701815080931701811171
:10113000A9CF60910D0170910E0180910F019091E6
:10114000100148813ADC80911401809317019ACFF5
:10115000462F682F80910D0190910E0138DD80910E
:101160000D0190910E01A0910F01B0911001810F1E
:10117000911DA11DB11D80930D0190930E01A093AF
:101180000F01B09310018091110190911201811B08
:1011900091099093120180931101892B29F41092E7
:1011A0001301FF24F3944BCFF12C49CF1BB815B892
:1011B0008BEF8AB98FEF84B914B883E087B99EEFBB
:1011C00098B985BDA6D878947AD779D7FDCFF89409
:0211D000FFCF4F
:0211D2005AFFC2
:00000001FF
